:100000000000000000006D28F100030EF20004085B
:10001000F3000A08F4008A01831203130B1F3C2823
:100020000B1A8B1C1B28781B1928E510C930DD23FF
:1000300066240B128B10831603138C1E2528831243
:1000400003138C1E252847208C12831603130C1CC7
:100050003C28831203130C1C3C28D203031D3528B3
:1000600065171930D20002308906101013308E0047
:100070007A308F0010140C108312031374088A0056
:1000800073088400720E8300F10E710E0900831252
:1000900003131819F814760884001A08C4008000A5
:1000A000F60AFD0A981C57281812181678150D30F4
:1000B0004406031965281B304406031978160319F2
:1000C00065287608633A031D0800831603138C1213
:1000D000831203131812F815080083120313FD018D
:1000E000CD01CE01D001FC01F8015330F600903073
:1000F000F7008316031382309F002F3085000330F2
:10010000860098308700F83089000030880081012F
:10011000B101B201BD01BE0183120313023086009A
:100120000730890081309F008B0107148714071561
:1001300009109801981718168316031398011815BB
:1001400098161F309900831203130B30F5003130DD
:10015000900013308E007A308F001930D200E510F5
:100160000C307724DD266624CF26091409151930B2
:10017000FA005930FB005B226624DD268618DC2855
:100180000030A6004530A5001630A4000630A300BC
:100190000430A2000330A1001130A0009030A7006D
:1001A00066242F2566240826662409101930FA00D3
:1001B0000030FB005B2266241730FA000030FB00A1
:1001C0005B2209147B2266240911DD260E243824C3
:1001D00053240915DD26E5141130DD233230DD23EB
:1001E0004330DD23B830DD236530DD230730403870
:1001F00054240030803854247630DD23DD267817EF
:100200000B16831603130C14831203138B170B178F
:10021000F80178125330F600FD0118168316031307
:100220008C1683120313E5140430890600002D2672
:10023000003040385424003080385424C1262F2503
:100240000910DD26D626F81D74291812831603130B
:100250008C1283120313E5103C2966247D08F900F3
:100260005B236D2442307F2475307F2466307F24E9
:1002700020307F24252366245330F60084000008B4
:10028000C40045304406031D4C29E514F816C92264
:10029000F8120430FC06742955304406031D542915
:1002A000F8116C23F815742948304406031D5B29A6
:1002B0001030FC0674294C304406031D6329422289
:1002C0000830FC06742957304406031D69294C2266
:1002D000742952304406031D6F29552274295A305F
:1002E0004406031D74295722C4017812651F76291C
:1002F0006513E514013089069F111F129F12C12654
:10030000E5126512AB23E516651233220130403841
:1003100054241E3080385424B324C126E5126512BB
:10032000013089069F151F129F12C126AB23023090
:1003300040385424183080385424E5126512E513EF
:10034000B324C126013089069F111F169F12C126B2
:10035000AB23033040385424183080385424E5123D
:100360006516E513B324C1266512831603133708F7
:10037000B1003808B2000030B3000B30B4005A2688
:10038000831203130430403854245F30B600043025
:100390004038542436088038542400305724B3267B
:1003A000B60BC72983160313BB013C088312031342
:1003B000003A0319E729B6000430403854243608BF
:1003C000803854243C305724B326B60BDC29053042
:1003D000403854240030803854246530DD23763092
:1003E000DD23063040385424183080385424370830
:1003F0008B133F238B17073040385424003080384C
:1004000054248730DD230227073040385424183025
:100410008038542438083F2301308906E510233002
:100420007724752289229522A122AD22B922422267
:10043000722447227224263077247C08103903194D
:10044000232A6D247B2266240914F81D13295330B6
:10045000F600FD01C401F8111816831603138C165B
:10046000831203131329831603130310B10DB20D66
:10047000B10DB20D831203130800DF30DD233708FE
:100480003F230800E230DD2338083F230800E53031
:10049000DD2337083F230800E5101830FA0000304C
:1004A000FB005B226624E5140800E510080000004C
:1004B0000800000008006222FF39031908007724B1
:1004C000FB0A5B2A831203177A088F007B088D00D2
:1004D000831603178C170C140000000083120317F7
:1004E00000000C0883120313080083120313C401D5
:1004F0002F2572240800C40166241730FA005030FA
:10050000FB005B2266247C120800C4014130772482
:100510000800E51265128522313077243D307724BA
:100520009F111F129F12C126C42AE512651285224F
:10053000323077243D3077249F151F129F12C12639
:10054000C42AE51265128522333077243D307724A2
:100550009F111F169F12C126C42AE512651285221B
:10056000343077243D3077249F151F169F12C12603
:10057000C42AE51265128522353077243D30772470
:100580009F111F129F16C126AB23B3247224C401EE
:100590000800E514053040385424003080385424D5
:1005A0006530DD2306304038542418308038542418
:1005B000063040385424183080385424F9018030F3
:1005C000CB005330F600F60A760884000008C40019
:1005D000AC00EB2331304406031DF02A4B08F9042C
:1005E0000310CB0C031CE32A7908B700F726C401DB
:1005F00008001A087812F8115330F600C401831667
:1006000003138C1683120313181644080319052BC1
:100610001812831603138C1283120313F8191B2B61
:100620004408AC001B3A031978160319202B2C0838
:10063000EB23F81DFE2A83120313F811C4010800EE
:100640005330F600C401F8110800CC017D08CB003E
:100650005330F600760884000008C500F60A7724B7
:100660000D30450603193C2BCC0ACB0303193C2B58
:100670002A2B72244C083F235330F6000800C50093
:10068000F900831603130830A2008312031303102A
:10069000F90D031C303003183130AC007724831679
:1006A0000313A20383120313031D472B3D30AC0039
:1006B00077244508F900790E0F39F63E0318073EF6
:1006C0003A3E772479080F39F63E0318073E3A3E42
:1006D0007724683077240800E510A830DD236624ED
:1006E000E5140530403854240030803854249830C4
:1006F000DD23073040385424003080385424F92258
:10070000073040385424003080385424781A0800C8
:10071000CB015330F600760884000008F60A8312F5
:100720000313C5000F30C5050310C50DC50DC50D5C
:10073000C50D760884000008F60A0F394507C50084
:100740004B08203E840045088000CB0ACB1D8B2B34
:100750000826DD2608008312031300001F14AC26B0
:100760001F15E5131F19B22B831203131E088316DE
:100770000313B100B5001E08B200B60083120313C4
:10078000E51ED22B831603130230B3000030B400F1
:100790007A26B11FD22B83120313E5178316031396
:1007A000B109B209C126831603133508B70036080C
:1007B000B800831203131F10080083120313B6003E
:1007C00036089424AC00B60AFF39031908002C0837
:1007D0007724E02B08008B138A11AD010A16002044
:1007E0000A125724AD0A0A1600200A125724AD0A2D
:1007F0000A1600200A125724AD0A0A1600200A120F
:100800005724AD0A0A1600200A125724AD0A0A1608
:1008100000200A125724AD0A8B1708001B24503001
:10082000F22626245030F2262A245030F22638248C
:100830005030F2260800183083160313930000305E
:100840009400831203132830940008000711CF2668
:1008500007150800213054249030542405305424C6
:100860001330542420305424BA260C305424080069
:1008700000304F2400304D24083054240930AA00A1
:100880006030AB0000305724AB0B422CAA0B402C3D
:1008900000304F2400304D2408008038542C40385C
:1008A000542C0D30542C0C30871000000000071021
:1008B0000000930000008C1D5B2C8C1100000714BD
:1008C00000008714080077246624080083120313AD
:1008D0000D307F240A307F2408008312031309306F
:1008E0007F240800831203133B307F240800831207
:1008F0000313AC00E518EB23E51C7F2408008312EA
:10090000031364000C1E822C990008008312031349
:10091000B60036089424AC00B60AFF390319080063
:100920002C087724892C0800831203178D00831666
:1009300003178C130C14831203170C088312031370
:100940000800640075080319AF2C0C1CAF2C1010A4
:10095000F50BAB2C00340C100B308F0010148C1ED8
:10096000A12C1A080800831603133108AF003208BF
:10097000B0002F0EF038A500A507E23EA600323EDB
:10098000A8002F080F39A607A607A807E93EA70069
:10099000A707A707300E0F39A707A807A70DA80DAF
:1009A000A809A80D30080F39A807A50D0730A40025
:1009B0000A30A807A703031CD92CA707A603031C0A
:1009C000DD2CA607A503031CE12CA507A403031C2B
:1009D000E52C83120313E51E112D2B30E51B2D3062
:1009E0007724831603132508031DFB2C831203139E
:1009F00020307724FF2C83120313303E7724831694
:100A000003132608303E77242E30772483160313F1
:100A10002708303E7724831603132808303E7724B6
:100A20000800651E182D831603132408303E772412
:100A3000831603132508303E7724831603132608F4
:100A4000303E7724831603132708303E772483161D
:100A500003132808303E77242030772408008312BF
:100A60000313220E0F39303E772422080F39303E0F
:100A700077242F307724210E0F39303E7724210838
:100A80000F39303E7724E5182030E51C2F307724CD
:100A9000E518522D200E0F39303E772420080F39EB
:100AA000303E772420307724240E0F39031D5A2D31
:100AB00020305B2D303E772424080F39303E7724D8
:100AC00048307724250E0F39303E772425080F391A
:100AD000303E77244D307724260E0F39303E772470
:100AE00026080F39303E7724533077240800782DBC
:100AF000792D7A2D7B2D7C2D7D2D7E2D7F2D802DAA
:100B0000812D822D832D842D852D862D872D882D59
:100B1000892D8A2D8B2D0800831686138312861744
:100B20000617772586137725061308008316861384
:100B300083128613061777258617080083168613F7
:100B40008312861377250617772506130800831668
:100B50008613831286177725061777250613080054
:100B60008316861783127725061777250315861BAC
:100B7000031106130800D2257725DB257725080009
:100B80008617831603130000861783120313772535
:100B900008008316031386138312031300008613C1
:100BA0007725080006178316031300000617831223
:100BB0000313772508008316031306138312031308
:100BC000061377250800C8010830CA00C025D225C1
:100BD000861FEB2DEE2D0310C80DF22D0310C80D4E
:100BE000C80AF22DDB25CA0BE72D0800C700083024
:100BF000CA000310C70D031CFE2D022EC925BB25FC
:100C0000C025052EC025BB25052ECA0BF92D0800D1
:100C10009625C8268C25D030F625B025C601460875
:100C2000F625B0252608F625B0252508F625B02599
:100C30002408F625B0252308F625B0252208F62538
:100C4000B0252108F625B0252008F625B0259030DE
:100C5000F625A7259625C82608009625AC268C25BE
:100C6000D030F625B025C6014608F625B025D1308E
:100C70008C25D130F625A725E3259E254808A6001A
:100C8000E3259E254808A500E3259E254808A400E5
:100C9000E3259E254808A300E3259E254808A200D9
:100CA000E3259E254808A100E3259E254808A000CD
:100CB000962508000310B901BA011030A100B20D49
:100CC000B10DBA0DB90D33083902031D692E340870
:100CD0003A02031C712E3408BA023308031CB30F06
:100CE000B902BC0DBB0DA10B5F2E3B08B1003C0847
:100CF000B20008008316031303103408B20233084D
:100D0000031C330FB1020800A3260310C00CBF0C54
:100D1000031C902E3908BB070318BC0A3A08BC070D
:100D2000BC0CBB0CBE0CBD0CC10B862E08004210C7
:100D30003908BB070318BC0A031842143A08BC0759
:100D40004218031408001030C1003C08C0003B08E2
:100D5000BF00BC01BB0108000130B3000130B4008A
:100D60001430B500EB2E0130B3000130B400503028
:100D7000B500EB2E0130B3000430B4003230B500C2
:100D8000EB2E0130B3002030B400CC30B500EB2E98
:100D90000130B3005030B4000130B500EB2E02300A
:100DA000B3007730B4000130B500EB2E0430B3004F
:100DB0003130B4000130B500EB2E1030B3000E30EE
:100DC000B4003830B500EB2E2030B3002830B4002A
:100DD000DA30B500EB2EB50BEB2EB40BEB2EB30BCC
:100DE000EB2E0800A900BA26A90BF32E08008C25CB
:100DF0004230F625AC26B0253709F625AC26A725C6
:0E0E000096250800D00A5008B800080000002F
:102000002C087F39B9000030BA00BC000630BB0094
:1020100006308A00842610308A001A30B00003107F
:102020003E088A073D0803102D0703188A0AB007E7
:1020300003188A0A82070034003400340034003464
:1020400000340034003400340034003400340034F0
:1020500000340034003400340034003400340034E0
:1020600000340034003400340034003400340034D0
:1020700000340034003400340034003400340034C0
:1020800000340034003400340034003400340034B0
:1020900000340034003400340034003400340034A0
:1020A0000034003400340034003400340034003490
:1020B0000034003400340034003400340034003480
:1020C0000034003400340034003400340034003470
:1020D0000034003400340034003400340034003460
:1020E0000034003400340034003400340034003450
:1020F0000034003400340034003400340034003440
:10210000003400340034003400340034003400342F
:10211000003400340034003400340034003400341F
:10212000003400340034003400340034003400340F
:1021300000340034003400340034003400340034FF
:1021400000340034003400340034003400340034EF
:1021500000340034003400340034003400340034DF
:1021600000340034003400340034003400340034CF
:1021700000340034003400340034003400340034BF
:1021800000340034003400340034003400340034AF
:10219000003400340034003400340034003400349F
:1021A000003400340034003400340034003400348F
:1021B000003400340034003400340034003400347F
:1021C0000034003400345F34003400340034003410
:1021D0000734003407340034003414347F341434AA
:1021E0007F341434003424342A347F342A341234B3
:1021F000003426341634083434343234003476341F
:102200004934553422345034003400340034053419
:1022100003340034003400341C342234413400349C
:1022200000340034413422341C340034003414347B
:1022300008343E34083414340034083408343E344E
:10224000083408340034003450343034003400345E
:1022500000340834083408340834083400340034B6
:1022600060346034003400340034203410340834D6
:102270000434023400343E345134493445343E345D
:102280000034003442347F3440340034003442346B
:1022900061345134493446340034213441344534B6
:1022A0004B34313400341834143412347F34103445
:1022B00000342734453445344534393400343C3413
:1022C0004A344934493430340034013401347934E7
:1022D000053403340034363449344934493436340F
:1022E000003406344934493429341E34003400346F
:1022F0003634363400340034003400345634363446
:1023000000340034003400340834143422344134AE
:102310000034143414341434143414340034413478
:10232000223414340834003400340234013451347B
:102330000934063400343E344134493455345E3473
:1023400000347E341134113411347E3400347F343F
:10235000493449344934363400343E34413441340C
:102360004134223400347F344134413422341C342B
:1023700000347F34493449344934413400347F34A3
:10238000093409340934013400343E3441344934C9
:1023900049343A3400347F340834083408347F3404
:1023A0000034003441347F3441340034003420346C
:1023B000413441343F34003400347F340834143421
:1023C0002234413400347F3440344034403440348B
:1023D00000347F3402340C3402347F3400347F34D0
:1023E0000434083410347F3400343E3441344134F2
:1023F00041343E3400347F3409340934093406341E
:1024000000343E344134513421345E3400347F345E
:1024100009341934293446340034463449344934B3
:10242000493431340034013401347F34013401340F
:1024300000343F344034403440343F3400341F349F
:102440002034403420341F3400343F3440343C3492
:1024500040343F3400346334143408341434633467
:1024600000340734083470340834073400346134DD
:102470005134493445344334003400347F344134DA
:10248000413400340034023404340834103420342D
:1024900000340034413441347F3400340034043497
:1024A00002340134023404340034403440344034C3
:1024B00040344034003400340134023404340034F5
:1024C00000342034543454345434783400347F3459
:1024D0004834443444343834003438344434443494
:1024E00044342034003438344434443448347F3461
:1024F00000343834543454345434183400340834E8
:102500007E340934013402340034083454345434F1
:1025100054343C3400347F34083404340434783484
:102520000034003444347D344034003400342034EA
:10253000403444343D34003400347F341034283483
:10254000443400340034003441347F3440340034A7
:1025500000347C34043418340434783400347C344B
:102560000834043404347834003438344434443483
:102570004434383400347C3414341434143408347F
:10258000003408341434143418347C3400347C346B
:102590000834043404340834003448345434543493
:1025A00054342034003404343F3444344034203430
:1025B00000343C344034403420347C3400341C3407
:1025C0002034403420341C3400343C34403438341B
:1025D00040343C34003444342834103428344434F7
:1025E00000340C345034503450343C3400344434CF
:1025F000643454344C3444340034003408343634B5
:10260000413400340034003400347F34003400346A
:102610000034003441343634083400340034083493
:1026200008342A341C340834003408341C342A3466
:06263000083408340034F8
:102E00002034503449344334313436344634383441
:102E100037343734203461347634653463342034C5
:102E200062346F346F3474346C346F3461346434AE
:102E300065347234203451343D34313430344D34BF
:102E400068347A340A340D3420344D3450344C34E0
:102E50004134423420347634653472347334693406
:102E60006F346E34203438342E34363433340A34EC
:102E70000D34203450346C346134743469346E341D
:102E800065342034313436344634383437343734CA
:102E9000203432343034313432340A340D34003496
:102EA0000A340D343C3448343E3465346C34703468
:102EB0000A340D343C3431343E3443346F346E3490
:102EC0007334693467346E346534203431340A34F1
:102ED0000D343C3432343E3443346F346E34733406
:102EE000693467346E346534203432340A340D3436
:102EF0003C3433343E3443346F346E347334693489
:102F000067346E346534203433340A340D343C3441
:102F10004C343E34653463347434753472346534FF
:102F200020345034433446340A340D343C34453470
:102F30003E346334723469347434753472342034FA
:102F40005034433446340A340D343C3455343E3422
:102F500070346434613474346534203452345434FD
:082F600043340A340D3400343F
:1030000020344C34453443345434553452344534EC
:1030100020344D3473346734203465346E342034B6
:1030200046344C34413453344834203464346534A9
:103030007034753469347334203430347834313436
:103040003834303430340A340D3420345034613460
:1030500067346534203420343D3420342034203427
:1030600020342034203420342034203420342034C0
:1030700020342034203420342034203420342034B0
:10308000203420342034203420340A340D342034C9
:103090005034613467346534203420343D34203476
:1030A0002034203420342034203420342034203480
:1030B0002034203420342034203420342034203470
:1030C00020342034203420342034203420340A3476
:1030D0000D34203450346134673465342034203466
:1030E0003D34203420342034203420342034203423
:1030F0002034203420342034203420342034203430
:10310000203420342034203420342034203420341F
:1031100020340A340D34203450346134673465343B
:10312000203420343D3420342034203420342034E2
:1031300020342034203420342034203420342034EF
:1031400020342034203420342034203420342034DF
:103150002034203420340A340D3420345034613487
:1031600067346534203420343D3420342034203416
:1031700020342034203420342034203420342034AF
:10318000203420342034203420342034203420349F
:10319000203420342034203420340A340D342034B8
:1031A00032343334343435343634373438343934D3
:1031B00030343134323433343434353436343734D3
:1031C00038343934303431343234333434343534BF
:1031D00036343734383439343034313432340A34D4
:0431E0000D34003476
:10320000203449346E3469347434203452345434A4
:10321000433420347034613472342034643465347F
:1032200066346134753474340A340D3420346134B6
:10323000753478342034763461346C3465347534C4
:1032400072347334203464346534663469346E34D3
:10325000693465347334203465346E342034643416
:103260007534723420342E342E340A340D34203424
:10327000643461346E34733420346C3465342034F7
:10328000703472346F346734723461346D346D3439
:10329000653420346334613472342034523442341F
:1032A00031343D34303420342E342E340A340D344D
:1032B00000342034563465347234733469346F34D6
:1032C0006E3420342034583450344F345234543413
:1032D0002D3441347234633468346F34733434348D
:1032E0003334693474342034523446344F346234C5
:1032F000613473346934633420340A340D34203437
:1033000065346E3420344D3450344C3441344234BE
:103310002034313430343034253420346134733443
:103320006D3420347234653476342034323436349B
:103330002F34303432342F34323430343134313469
:10334000203420340A340D34203450346C34613449
:10335000743469346E3465345F3431343634463411
:103360003834373437345F346E346F346B34693407
:1033700061345F34583470346F34723474345F3471
:1033800041347234633468346F3473345F343134AD
:10339000323430343234323436342E34613473348F
:1033A0006D3420340A340D34003431343234333443
:1033B00034343534363437343834393430343134C5
:1033C00032343334343435343634373438343934B1
:1033D00030343134323433343434353436343734B1
:1033E000383439343034313432340A340D34003422
:02400E00323D41
:104200003134363446343834373437342034773424
:10421000203462346F346F3474346C3464347234E8
:104220000034323436342F34303432342F34323494
:10423000303431343234203432343034483433344E
:104240003034433448343034203420342034203463
:104250002034203420342034203455344E34493432
:10426000543400344334483431342034203420343E
:10427000203420342034203450344F3449344E34E8
:1042800054345334003443344834323420342034EA
:104290002034203420342034203450344F344934F6
:1042A0004E34543453340034433448343534203499
:1042B0002034203420342034203450344F344934D6
:1042C0004E34543453342034003450344F34523448
:1042D000543453342034383442342034503443344A
:1042E0004634383435343734343400344534433488
:1042F00052342034203420342034203420342034EC
:1043000020342034203420342034203400344C3401
:1043100045344334203420342034203420342034B5
:10432000203420342034203420342034203400340D
:104330004D3441344A3420344434533431343334EA
:1043400030343734203420342034203420342034A6
:10435000413441344D344D344A344A34573457345F
:10436000483448344D344D3453345334203420349D
:10437000203420342034203420342034203420349D
:10438000203420342034203420342034203420348D
:10439000003449344E345434453452345534503456
:1043A000543420345234423430342E342E342E34AB
:1043B0002E340034503443344634203400344534F1
:1043C0003D3400344C343D34003452343D340034F8
:00000001FF
